S02B0000443A2F7573722F6665617365722F736F6674776172652F4F70656E424C542F5461726765742F44657D
S1132000E801002071210000BD270000BD27000069
S1132010BD270000BD270000BD270000BD2700002C
S1132020BD270000BD270000BD270000BD2700001C
S1132030BD270000BD270000BD270000A927000020
S1132040BD270000BD270000BD270000BD270000FC
S1132050BD270000BD270000BD270000BD270000EC
S1132060BD270000BD270000BD270000BD270000DC
S1132070BD270000BD270000BD270000BD270000CC
S1132080BD270000BD270000BD270000BD270000BC
S1132090BD270000BD270000BD270000BD270000AC
S11320A0BD270000BD270000BD270000B933000094
S10F20B0BD270000BD270000EE11AA555A
S11320BC2E498D462E492F480A1A04D081F30988DB
S11320CC022282F314882C482C492D4A00F039F84A
S11320DC2C482D492D4A00F034F82D482D492E4A10
S11320EC00F02FF82D482E492E4A00F02AF82E48DD
S11320FC2E492F4A00F025F82E482F492F4A00F07C
S113210C20F82F482F49002200F026F82E482F499A
S113211C091A082903DB00220260043001602048FC
S113212C2049884205D00268043003B4904703BCAC
S113213CF7E700208646EC4600200021244A90470D
S113214CFEE7884207D0521A05D0037801300B7091
S113215C0131013AF9D17047884202D00270013042
S113216CFAE770471B481C490160A1E7E80100200D
S113217CE8010020E8010020784200000000002063
S113218C08000020E8210000E82100004042000083
S113219C78420000000000200000002040420000B3
S11321AC4042000040420000404200004042000017
S11321BC40420000404200004042000078420000CF
S11321CC080000206800002068000020E8000020BF
S10F21DC7524000008ED00E00020000065
S11321E810B504464FF48843C4F20803DB6A13F0BD
S11321F8040F0CD04FF48840C4F2080043F2B5230E
S1132208C0F20003984720704FF0010010BD4FF052
S1132218000010BD30B586B06C4644F24025C0F2CB
S113222800050FCD0FC495E8030084E803004FF4BC
S11322384240C0F202004FF0010142F6D134C0F22C
S11322480004A0474FF002004FF006014FF00402CB
S11322584FF0010343F2DD05C0F20005A8474FF033
S113226802004FF007014FF001024FF00003A847A6
S11322784FF40C50C0F204004FF00101A0474FF096
S11322880300C0F212004FF0020142F69973C0F243
S1132298000398474FF4AA55C0F2160528464FF094
S11322A8010142F6CD13C0F20003984728464FF0C7
S11322B80101A0474FF0000506A941F8185D4FF445
S11322C88844C4F208042046694643F25523C0F200
S11322D800039847204629464FF4165243F2B51393
S11322E8C0F2000398474FF0030363654FF00403FB
S11322F8636320464FF0050143F21923C0F200033B
S1132308984706B030BD00BF00B540F24D03C2F295
S113231800031B78D3B940F20800C2F2000042F26D
S1132328E913C0F20003984701284ED140F24D0347
S1132338C2F200034FF001021A7040F24C03C2F2D9
S113234800034FF000021A705DF804FB40F2080322
S1132358C2F2000340F24C02C2F20002107800F10B
S11323680100181842F2E913C0F200039847012843
S11323782BD140F24C03C2F200031A7802F1010295
S1132388D2B21A7040F20803C2F200031B789342D7
S11323981BD140F24D03C2F200034FF000021A7041
S11323A840F20803C2F200035B78FF2B0DD140F220
S11323B80803C2F200039B783BB942F22573C0F2CA
S11323C8000398474FF0B90398475DF804FB00BF32
S11323D862B6704700B54FF42040C4F2080043F2D7
S11323E89D43C0F2000398475DF804FB10B542F220
S11323F89D73C0F200039847044640F25003C2F2AA
S113240800031B68C31AB3F5FA7F2ED340F24E03B8
S1132418C2F200031B7893B940F24E03C2F20003E0
S11324284FF001021A704FF42040C4F208004FF034
S1132438000143F2F533C0F20003984710E040F27C
S11324484E03C2F200034FF000021A704FF420400A
S1132458C4F20800114643F2F533C0F2000398476A
S113246840F25003C2F200031C6010BD00B581B0F5
S113247842F6A503C0F20003984748F2FC13C0F6DD
S1132488E0731B681B0E14D14AF20C03C4F20C034C
S11324981A6822F070021A6046F22003C4F20C0390
S11324A81A6822F060421A601A6862F060621A6060
S11324B801E0032B22D846F22003C4F20C031A6865
S11324C822F4FC521A6048F24002C4F20C024FF0A3
S11324D80003136048F24402C4F20C02136048F289
S11324E85802C4F20C02136048F26002C4F20C02EF
S11324F8136048F27802C4F20C021360684643F28F
S1132508C523C0F2000398479DF80030012B17D16A
S11325189DF801303BB948F24003C4F20C031A6831
S113252842F002021A609DF80130012B9FBF48F265
S11325384403C4F20C031A6842F0010298BF1A60FB
S113254848F2F013C0F6E0731A684BF6FF13C4F6AA
S11325588A439A422FD848F24403C4F20C031A68F7
S113256842F490421A6048F2B412C0F6E07211685C
S1132578C1F3062110681568146804F07F0405F493
S1132588FE42224300F07F0042EA004242EA01612F
S113259842F23402C4F20002116048F2C812C0F6D2
S11325A8E072116844F22C02C4F2000211601A6845
S11325B822F490421A604FF000004FF001010A46DD
S11325C842F62173C0F2000398474FF40043C4F263
S11325D80C031A6C42F00F021A645A6C6FEA124226
S11325E86FEA02425A644FF44070C0F204004FF09C
S11325F8000142F6D134C0F20004A0474FF49850C9
S1132608C0F204004FF00001A0474FF44C50C0F250
S113261804004FF00001A0474FF42240C0F202002A
S11326284FF00001A0474FF40070C0F202004FF0D1
S11326380001A0474FF49050C0F202004FF000018F
S1132648A0474FF40850C0F202004FF00001A04721
S11326584FF44850C0F202004FF00001A0474FF475
S1132668E440C0F202004FF00001A0474FF40240DA
S1132678C0F202004FF00001A0474FF43240C0F20C
S113268802004FF00001A0474FF46240C0F202007C
S11326984FF00001A0474FF47240C0F202004FF01F
S11326A80001A0474FF45240C0F202004FF000016D
S11326B8A0474FF001004FF009014FF0050203460F
S11326C843F2DD04C0F20004A0474FF001004FF0CC
S11326D8020143F2C103C0F20003984742F2DD331A
S11326E8C0F20003984742F24173C0F200039847CE
S11326F842F2D933C0F20003984742F21D23C0F2D4
S11327080003984742F2F535C0F2000542F211344D
S1132718C0F20004A847A047FCE700BF4EF210032C
S1132728CEF200034FF000021A60704740F25403DF
S1132738C2F200031860704700B54FF02000C0F2E1
S1132748040042F61953C0F20003984744F6D353E1
S1132758C1F26203A3FB0020C0F3971000F1FF301D
S11327684EF21003CEF2000358604FF46D42CEF2DD
S113277800024FF0E00182F823104FF00000986047
S11327884FF007021A6042F23573C0F2000398470B
S11327985DF804FB40F25403C2F200031868704762
S11327A840F25403C2F200031A6802F101021A60EB
S11327B8704700BFFEE700BF4FF40043C4F20C03A8
S11327C8DB6A03F47053B3F5805F48D0B3F5005F58
S11327D803D0B3F5006F0CD105E040F20003C2F258
S11327E800031868704740F20403C2F20003186833
S11327F870474FF40043C4F20C03DB6803F4E0634E
S1132808B3F5007F19D004D80BB3B3F5807F23D177
S113281818E0B3F5806F25D0B3F5A06F03D0B3F5F6
S1132828407F19D104E04FF47C50C0F2AB107047DC
S113283849F68070C0F2D50070474DF6C000C0F26A
S1132848A70070474CF6C070C0F26A00704744F2A3
S11328584020C0F20F0070474FF0000070474FF45B
S11328680040704746F64070C0F24010704700BF01
S113287800B542F2C173C0F2000398474FF4004315
S1132888C4F20C035B6803F00F0320FA03F040F270
S11328985803C2F2000318605DF804FB704700BFD8
S11328A84FF40040704700BF40F20003C2F2000337
S11328B8186870474FF00003C4F20C035B6803F018
S11328C80702032A0CD8DFE802F00202070723F004
S11328D8070343F0010303E023F0070343F0030372
S11328E84FF00002C4F20C0253607047B0FA80F053
S11328F8C0B2C0F11F0070474FF00003C4F20C03CC
S11329085B684DF6FF32CFF60B72821842F2FF3144
S1132918C0F2F4018A420BD803F00702A2F10202C2
S1132928012A23F0070394BF43F0030343F0010390
S11329384FF41052C0F2F402904209D803F007028F
S1132948A2F10202012A23F0070398BF43F002030D
S11329584FF00002C4F20C025360704749F68070CD
S1132968C0F2D500704700BF00B54FF40043C4F26D
S11329780C039B6A4FEA400023FA00F000F00300BE
S113298802280AD003280FD0012816D142F6A90339
S1132998C0F2000398475DF804FB42F6B103C0F2A5
S11329A8000398475DF804FB42F67903C0F200037C
S11329B898474FEA50005DF804FB4FF000005DF8BB
S11329C804FB00BF10B50C46C0F3031303F1FF3337
S11329D8032B00F2F780DFE803F0021231A808465F
S11329E842F6F503C0F2000398474FF40043C4F2DB
S11329F80C039A6822F00F021043986010BD42F647
S1132A08BD03C0F200039847204642F6F503C0F21E
S1132A18000398474FF40043C4F20C035A6822F0A9
S1132A280F021043586042F67903C0F20003984736
S1132A3842F60113C0F20003984710BD41F2304337
S1132A48C0F20A0398422CD04FF03003C0F20C03B2
S1132A58984247D04FF48663C0F20803984240F086
S1132A68B1804FF40043C4F20C035B6D13F0010F03
S1132A7807D14FF40042C4F20C02136D13F0040F93
S1132A88FBD1204642F6F503C0F2000398474FF401
S1132A980043C4F20C039A6E22F00F0210439866A6
S1132AA810BD4FF40043C4F20C035B6D13F0010F27
S1132AB807D14FF40042C4F20C02136D13F0040F53
S1132AC8FBD1204642F6F503C0F2000398474FF4C1
S1132AD80043C4F20C039A6E22F0F00242EA00109A
S1132AE8986610BD4FF40043C4F20C035B6D13F0F9
S1132AF8010F07D14FF40042C4F20C02136D13F016
S1132B08040FFBD1204642F6F503C0F200039847B0
S1132B184FF40043C4F20C039A6EA0F1100022F49F
S1132B28407242EA00229A6610BD4FF4A863C0F2CC
S1132B381403984206D04FF4AA53C0F216039842DD
S1132B4840D11FE04FF40043C4F20C035B6D13F053
S1132B58010F07D14FF40042C4F20C02136D13F0B5
S1132B68400FFBD1204642F6F503C0F20003984714
S1132B784FF40043C4F20C031A6F22F0030210430B
S1132B88186710BD4FF40043C4F20C035B6D13F0D7
S1132B98010F07D14FF40042C4F20C02136D13F075
S1132BA8400FFBD1204642F6F503C0F200039847D4
S1132BB84FF40043C4F20C031A6F22F0300242EAC5
S1132BC80010186710BD00BF30B4C9B2C0F30323A6
S1132BD803F1FF33052B43D8DFE803F008363B1E27
S1132BE8250348F27802C4F20C0236E0C0F304303C
S1132BF848F20802C4F20C0206E04FF40044C4F29E
S1132C080C04236D1D42FCD102F1047200EBC202D4
S1132C184FEA8202116023E04FF0010548F258029E
S1132C28C4F20C0205E04FF0100548F26002C4F249
S1132C380C02C0F304304FF40043C4F20C035B6D80
S1132C4813F0010FE0D1D8E748F24402C4F20C02B1
S1132C5803E048F24002C4F20C02C0F30430D3E7A4
S1132C6830BC704700F00F0000F1FF30032842D851
S1132C78DFE800F0051B2E024FF0070070474FF401
S1132C880043C4F20C03D86A00F47050B0F5805FB6
S1132C9834D0B0F5005F05D0B0F5006F0CBF042048
S1132CA8052070474FF0020070474FF40043C4F208
S1132CB80C03986A00F00300022822D0032804D0E9
S1132CC801280CBF0320012070474FF0060070470D
S1132CD84FF40043C4F20C03986A00F00C00022875
S1132CE812D0032804D001280CBF03200120704708
S1132CF84FF0060070474FF0000070474FF0030094
S1132D0870474FF0020070474FF00200704700BF51
S1132D1800B500F47810B0F5402F7AD014D8B0F587
S1132D28802F42D005D848B3B0F5003F40F0EF807B
S1132D382BE0B0F5002F48D0B0F5202F57D0B0F5D0
S1132D48C02F40F0E48037E0B0F5A01F00F0958074
S1132D5807D8B0F5602F6ED0B0F5901F40F0D7803B
S1132D6882E0B0F5C01F00F0AC80B0F5D01F00F0D1
S1132D78C780B0F5B01F40F0CA8090E042F2C1733A
S1132D88C0F2000398475DF804FB42F2C173C0F235
S1132D98000398474FF40043C4F20C039B6803F004
S1132DA80F0320FA03F05DF804FB42F67903C0F23E
S1132DB8000398475DF804FB4FF0000042F67113D6
S1132DC8C0F2000398475DF804FB4FF0000042F698
S1132DD87113C0F2000398474FF40043C4F20C0384
S1132DE89B6E03F00F0320FA03F05DF804FB4FF029
S1132DF8000042F67113C0F2000398474FF40043F1
S1132E08C4F20C039B6EC3F3031320FA03F05DF8BA
S1132E1804FB4FF0000042F67113C0F20003984718
S1132E284FF40043C4F20C039B6EC3F3012320FA4E
S1132E3803F05DF804FB4FF0000042F67113C0F292
S1132E48000398474FF40043C4F20C039A6EC2F38C
S1132E58012220FA02F0DB6F03F0070303F10103F8
S1132E68B0FBF3F05DF804FB4FF0010042F6711378
S1132E78C0F2000398475DF804FB4FF0010042F6E6
S1132E887113C0F2000398474FF40043C4F20C03D3
S1132E981B6F03F0030320FA03F05DF804FB4FF003
S1132EA8010042F67113C0F2000398474FF400433F
S1132EB8C4F20C031B6FC3F3011320FA03F05DF88B
S1132EC804FB4FF00400C0F2180042F66D43C0F250
S1132ED800039847072808D008280DD142F2C17387
S1132EE8C0F2000398475DF804FB42F66513C0F28C
S1132EF8000398475DF804FB4FF000005DF804FBFD
S1132F0842F66513C0F2000398475DF804FB4FF0DE
S1132F1800005DF804FB00BF10B5C9B2D2B20428A2
S1132F2835D8DFE800F0120D170308004FF001044C
S1132F384FF0020012E04FF010044FF020000DE0B3
S1132F484FF040044FF0800008E04FF480744FF4D1
S1132F58007003E04FF004044FF0080069B14FF427
S1132F680043C4F20C031C6262B14FF40042C4F281
S1132F780C02D36A1842FCD004E04FF40043C4F2B4
S1132F880C03186243F2A903C0F20003984710BD6A
S1132F9810B500F00F00012804D000287FD00328C2
S1132FA87DD83BE0A1F10201032978D8DFE801F0DC
S1132FB80210070B4FF000004FF004040CE04FF030
S1132FC80200044608E04FF003004FF0010403E058
S1132FD84FF001004FF003044FF001010A4642F696
S1132FE82173C0F20003984742F6BD03C0F2000300
S1132FF898474FF40043C4F20C035C6243F2A903FC
S1133008C0F20003984742F67903C0F200039847D8
S113301842F60113C0F20003984710BD022814BFFA
S11330280224002401F1FF31052938D8DFE801F032
S113303826031037371C4FF000004FF001010A46F1
S113304842F62173C0F2000398474FF0020217E0DA
S11330584FF001000146024642F62173C0F2000314
S113306898474FF001020BE040F60803C4F290338E
S11330784FF001021A604FF0030201E04FF0000222
S11330884FF40043C4F20C03996A02FA04F24FF0B5
S1133098030000FA04F421EA040414439C6210BDFA
S11330A84FF40043C4F20C03DA6A40F25C03C2F240
S11330B800031A80704700BF4FF4C043C4F20003F2
S11330C800EBC0004FEA80001A5822F003021143B3
S11330D819507047F0B4DAB16BB14FF0010505FA35
S11330E801F500EBC0044FEA840404F1804404F5BC
S11330F8C04425610CE04FF0010505FA01F500EB29
S1133108C0044FEA840404F1804404F5C0446561B2
S1133118072915D800EBC0044FEA840404F180445D
S113312804F5C04467684FEA81054FF00F0606FAB4
S113313805F627EA060602FA05F53543656016E042
S113314800EBC0044FEA840404F1804404F5C0444D
S1133158A7684FEA8105A5F120054FF00F0606FA86
S113316805F627EA060602FA05F53543A560DAB935
S11331786BB14FF0010303FA01F100EBC0004FEA11
S1133188800000F1804000F5C04001610CE04FF080
S1133198010303FA01F100EBC0004FEA800000F1DB
S11331A8804000F5C0404161F0BC704730B504462A
S11331B81546D9B94FF48043C4F2080398420BD09A
S11331C84FF48843C4F20803984204BF4FF4AA504A
S11331D8C0F216001BD103E04FF4A860C0F214003B
S11331E842F61953C0F20003984701464FEA4111C9
S11331F8B1FBF5F5A5F120054FEAC505236C13F0DD
S1133208010F03D1636C13F0040FFBD1E56030BDEB
S11332186FEA010303F0050341EA4301036C13F069
S1133228010F03D1436C13F0020FFBD141607047C7
S1133238C9B231B1436C002BFCD14FF001030364D4
S113324870474FF000030364704700BF70B504462D
S11332580D46036C13F0010F03D1636C13F0020FD6
S1133268FBD14FF00A03636020464FF0010143F29B
S11332783926C0F20006B04722682969EB680B4377
S113328869690B4322F01C02134323606968AA6826
S1133298204643F2B513C0F2000398472B686360D5
S11332A820464FF00001B04770BD00BF836813F09B
S11332B8200FFBD0C069C0B2704700BF4FF6D0736F
S11332C8CEF20F031A6902F03F0202709A6902F003
S11332D8F002DB69C3F3031313434370704700BF61
S11332E81F2AC4BF203A04314FF0010303FA02F243
S11332F8072924D8DFE801F004080C1014181C204E
S1133308036C1A4302647047436C1A43426470475F
S1133318836C1A4382647047C36C1A43C26470474F
S1133328036D1A4302657047436D1A43426570473B
S1133338836D1A4382657047C36D1A43C26570472B
S11333481F2AC4BF203A04314FF0010303FA02F2E2
S113335807292CD8DFE801F004090E13181D2227C9
S1133368036C23EA020202647047436C23EA0202F4
S113337842647047836C23EA020282647047C36C18
S113338823EA0202C2647047036D23EA020202655B
S11333987047436D23EA020242657047836D23EA4E
S11333A8020282657047C36D23EA0202C265704750
S11333B84FF42043C4F208034FF0FF325A6240F23C
S11333C86003C2F200031A6802F101021A6070472E
S11333D84FF00003036403654364436583648365B2
S11333E8C364C365436E002BFCD1704730B50B2909
S11333F83FD8DFE801F03A060B0F14191E23282DD5
S113340831354FF003034FF0010432E04FF003036A
S11334181C462EE04FF003034FF0000429E04FF060
S113342803034FF0020424E04FF027034FF0000495
S11334381FE04FF027034FF003041AE04FF0010395
S11334484FF0030415E04FF001034FF0020410E0BD
S11334584FF001031C460CE04FF001031C4608E042
S11334684FF007034FF0030403E04FF00F034FF04E
S113347803043AB121461A4643F2E923C0F2000391
S1133488984730BD21461A4643F24933C0F2000337
S1133498984730BD10B504464FF40043C4F20C03FA
S11334A89A6A22F003029A629A6A42F002029A62C3
S11334B89A6D42F004029A659A6E22F440729A66F2
S11334C89A6E42F440729A664FF000038362636E08
S11334D8002BFCD14FF0FF3363624FF46143CEF20B
S11334E800034FF000621A604FF00103A36241F633
S11334F80B7363604FF40043C4F20C034FF00002F3
S1133508DA67204643F2D933C0F20003984740F201
S1133518FF33A3604FF005032360636E002BFCD1D7
S11335284FF48073C0F21C03E360636E002BFCD17C
S11335384FF001036362A36210BD00BF00B50346E8
S113354802783AB14268107840B102F101025A6037
S11335585DF804FB436898475DF804FB4FF0FF30BF
S11335685DF804FB30B50446C8B2A16849B12368C4
S1133578626803F10105954208BF0020934238BFF1
S1133588C854E3682BB121686268914201D221468C
S11335989847236803F10103236030BDF0B515464D
S11335A801290BD40E464FF00004C7B22846394609
S11335B8FFF7D8FF04F10104B442F7D1F0BD00BF0E
S11335C800B510F0100F07D100F4007000280CBFEC
S11335D820203020FFF7E2FF5DF804FBA0F1410052
S11335E819288CBF00200120704700BFA0F161009A
S11335F819288CBF00200120704700BFA0F13000BB
S113360809288CBF00200120704700BF30B504464C
S11336180D46FFF7F3FF10B1A4F130000FE0204688
S1133628FFF7E4FF10B1A4F1570008E02046FFF7C4
S1133638D5FF10B1A4F1370001E04FF0FF30A842E4
S1133648A8BF4FF0FF3030BDA0F10903202814BFF4
S113365800200120042B98BF40F00100704700BFF0
S113366800F1010110F0030F11D010F8012B002A0A
S113367823D010F0030F0AD010F8012B002A1CD015
S113368810F0030F03D010F8012B002A15D02DE9F0
S113369870004FF001324FF0803350F8044BA4EB24
S11336A8020525EA04051D4000D1F6E7A0F104004F
S11336B870BC10F8012B002AFBD1A0EB0100704765
S11336C82DE9F04F87B007460C4603924FF00003EC
S11336D8036044F2582BC0F2000B44F26823C0F292
S11336E800030293C1E204F10104252904BF23461F
S11336F8002603D03846FFF735FFB6E2194613F81B
S1133708010B1C46A0F12002102A1CD8DFE802F0A5
S1133718091B1B0C1B1B1B0F1B1B1B121B151B1B29
S1133728180046F04006E9E746F08006E6E746F466
S11337380046E3E746F02006E0E746F01006DDE73A
S113374846F40076DAE72A2808D0A0F13002D2B28B
S1133758092A88BF4FF0000A11D920E0039B03F11E
S113376804000390D3F800A0BAF1000FBCBFCAF15B
S1133778000A46F01006487801F102040FE04FF001
S1133788000A0AEB8A0AA0F1300000EB4A0A13F88F
S1133798010B1C46A0F13002D2B2092AF1D92AEA57
S11337A8EA7A2E2818BF4FF000082DD120782A284D
S11337B80AD004F10104A0F13003DBB2092B88BF5D
S11337C84FF000080AD91DE0039B03F10402039299
S11337D8D3F80080607804F1020410E023464FF027
S11337E8000808EB8808A0F1300000EB480813F83B
S11337F8010B1C46A0F13002D2B2092AF1D9B8F162
S1133808000F01DB46F4807668280AD120786828FE
S113381803BF46F0080660780234013418BF46F046
S1133828040678287AD8DFE810F02E0279007900A7
S113383879007900790079007900790079007900B4
S113384879007900790079007900790079007900A4
S11338587900790079007900790079007900790094
S11338687900790079007900790079007900790084
S1133878790079008A007900790079007900790063
S11338887900790079007900790079007900790064
S11338987900790079007900790079007900790054
S11338A87900790079007900790079007900790044
S11338B87900790079007900790079007900790034
S11338C87900790079007900790079007900790024
S11338D879007900790079007900EE00790079009F
S11338E87900790079007900790079007900790004
S11338F890001A0179007900790079001A01790099
S1133908790079007900AB000201DB0079007900C5
S1133918B7007900110179007900F00040F26403DE
S1133928C2F200031D68002D00F09F81CDF80080CD
S113393803AB0193394632465346A84795E13846C6
S11339484FF02501FFF70EFE8FE1039B03F10402FC
S113395803921D780AF1FF3A304651463A46FFF77A
S11339682FFE38462946FFF7FDFD16F0100F00F02C
S11339787C814FF0200051463A46FFF70FFE74E170
S113398816F0080F039B03F1040203921B683A68BC
S113399814BF1A701A6068E1039B03F104020392CE
S11339A8D3F800904846FFF75BFE05468045ACBF58
S11339B80023012303EA1623002B18BF4546C5EB51
S11339C80A0A304651463A46FFF7FAFD002DCCD094
S11339D819F8011B3846FFF7C5FD013DF8D1C4E7C6
S11339E8039B03F1040203921B6806F08009B9F1F2
S11339F8000F14BF4FF023094FF0000946F48076F6
S1133A084FF0080869E046F4005643F2780343F29D
S1133A185809782808BF994616F0800F08BF4FF058
S1133A28000916F4807F18BF26F400761EE006F01D
S1133A388009B9F1000F14BF4FF030094FF00009A5
S1133A4816F4807F18BF26F400760FE016F4807F02
S1133A581CBF26F400764FF0000907D104E046F4B1
S1133A6880464FF0000901E04FF0000916F4804F3A
S1133A781DD0039B03F1040203921B6816F0040F84
S1133A8818BF1BB203D116F0080F18BFDBB2002B06
S1133A98BCBF5B424FF02D091ADB06F04002002A36
S1133AA818BF4FF0200916F0200F11D00EE0039B29
S1133AB803F1040203921B6816F0040F18BF9BB2AB
S1133AC806D116F0080F18BFDBB201E04FF02B093E
S1133AD816F4807F04D026F4007616F4807F01D192
S1133AE84FF00108A0F15800202870D8DFE800F052
S1133AF8196F6F6F6F6F6F6F6F6F6F6F156F6F6F7A
S1133B086F156F6F6F6F6F11196F6F6F6F156F6F21
S1133B1819004FF000050BBB5BE04FF0000553BBE9
S1133B2857E04FF00005002B53D04FF0000506F482
S1133B380052DDF808E032B103F00F011EF801006D
S1133B4804A9685405E003F00F011BF8010004A957
S1133B58685405F101051B09EDD13AE04FF0000561
S1133B6803F0070101F1300104AAA95405F1010584
S1133B78DB08F5D12DE04FF0000506F4004C4CF6B7
S1133B88CD4ECCF6CC4E6246A446144654B105F04C
S1133B980302032A01BF07A842192C2102F80C1CAE
S1133BA808BF013507AA5119AEFB03024FEAD20236
S1133BB802EB8200A3EB400303F1300301F80C3C51
S1133BC805F101051346002AE0D1644601E04FF0EF
S1133BD80005C5EB080828EAE878C8EB0A0AC5EB2B
S1133BE80A0AB9F1FF0F88BF0AF1FF3AB9F1000FC9
S1133BF801D00AF1FF3A16F4007F06D13046514647
S1133C083A46FFF7DDFC4FF0000AB9F1FF0F04D97B
S1133C18C9F307213846FFF7A5FCB9F1000F04D012
S1133C285FFA89F13846FFF79DFC304651463A461B
S1133C38FFF7C6FC4FF0300041463A46FFF7AEFCAA
S1133C48012D09D40DF11008454415F8011D384615
S1133C58FFF788FC4545F8D116F0100F05D04FF052
S1133C68200051463A46FFF799FC217800297FF451
S1133C783AADBB682BB13A6879688A423CBF0021E7
S1133C889954386801E04FF0FF3007B0BDE8F08F71
S1133C9810B504460B783BB1B0F1FF3F06D04B6832
S1133CA803F1FF334B6001E08B689847204610BD51
S1133CB82DE9F04F82468B4617469846099E4FF0E9
S1133CC8FF3900E0A94609F101055046FFF736FC23
S1133CD80446FFF7B9FC0028F4D12346B4F1FF3FAA
S1133CE808BF4FF0FF3500F09C8027F4C067002E12
S1133CF84EDD17F0800F0DD02B2C03D02D2C09D1BD
S1133D0847F4806709F102055046FFF717FC04469B
S1133D1806F1FF36302C14BF00230123002ED4BF34
S1133D28002303F00103002B32D047F4007706F197
S1133D38FF3605F101095046FFF700FC0446002E42
S1133D4820DD582814BF00230123782808BF43F036
S1133D580103BBB1B8F1100F14BF00230123B8F15C
S1133D68000F08BF43F0010363B127F4007706F19D
S1133D78FF3605F102095046FFF7E0FB04464FF011
S1133D88100851E0B8F1000F08BF4FF008084BE0E5
S1133D98B8F1000F08BF4FF00A08002ED8BF4FF043
S1133DA800090EDC15E047F4007706F1FF3608FB3E
S1133DB8090905F101055046FFF7C0FB044616B989
S1133DC807E04FF0000920464146FFF71FFC002892
S1133DD8E9DA20465146FFF75BFF17F4007F08BF76
S1133DE86FF001051DD017F0010F1AD1DBF8003070
S1133DF803F10402CBF800201B6807F49062B2F5C3
S1133E08906F08BFC9F1000917F0100F18BF83F8A5
S1133E18009006D117F0080F14BFA3F80090C3F858
S1133E2800902846BDE8F08F4D46B6E72DE9F04FDF
S1133E3885B001908A4604924FF0000BCDF808B083
S1133E484CF6CC49C0F6CC49544614F8015B002D15
S1133E5800F0DE81252D3BD02846FFF7F5FB08B995
S1133E6818E02C4604F101052078FFF7EDFB002843
S1133E78F7D101E00BF1010B0198FFF75FFB054651
S1133E88FFF7E2FB0028F5D128460199FFF700FF68
S1133E98A246D9E70198FFF751FB0646A84203D189
S1133EA80BF1010BA246CFE70199FFF7F1FE029A45
S1133EB8D2F1010338BF0023B6F1FF3F14BF002637
S1133EC803F00106002E18BF4FF0FF3202929FE163
S1133ED89AF801302A2B06BF0AF102044FF00108B0
S1133EE84FF000084FF000050CE04D4500F39081B9
S1133EF805EB8505A6F1300616EB450500F188812A
S1133F0848F02008274604F101043E78A2463046CA
S1133F18FFF774FB0028E8D1414608F02002002A84
S1133F2808BF6FF000454C2E05D17E7807F1020AD0
S1133F3848F044080EE0682E0CD17E78682E03BF42
S1133F4848F01008BE7807F1030A07F1020A18BFFF
S1133F5841F00808A6F12506532E00F25981DFE83E
S1133F6816F05400570157015701570157015701DB
S1133F785701570157015701570157015701570175
S1133F885701570157015701570157015701570165
S1133F985701570157015701570157015701570155
S1133FA85701570157015701570157015701570145
S1133FB85701570157015701570157015701570135
S1133FC85701570157015701330157015701570149
S1133FD857015701570157015701570157017000FD
S1133FE89F005701570157015701AA00570157016C
S1133FF857015701B500CD00D80057015701E30018
S1134008570128015701570133010198FFF796FA20
S11340180446252802D10BF1010B15E70199FFF796
S113402837FE029A131C18BF0123B4F1FF3F0CBFDB
S11340381C4643F00104002C08BF4FF0FF320292E3
S1134048E6E008F02003002B08BF012518F001045E
S113405801BF049B1A1D04921E6818BF0026002D78
S113406800F0D680002D13DD0198FFF767FAB0F150
S1134078FF3F06D1029B002B08BF4FF0FF3302938A
S1134088C6E00CB906F8010B0BF1010B013DEBD1AD
S1134098002C7FF4D9AE029B03F101030293D3E60B
S11340A848F080020095019804A94FF00A03FFF72D
S11340B8FFFD044692E048F080020095019804A9A7
S11340C84FF00003FFF7F4FD044687E018F0010FF2
S11340D87FF4BAAE049B03F1040204921B6818F03F
S11340E8100F18BF83F800B07FF4AEAE18F0080FB5
S11340F814BFA3F800B0C3F800B0A5E648F08002E6
S11341080095019804A94FF00803FFF7D1FD044670
S113411864E028F01E020095019804A94FF01003EA
S1134128FFF7C6FD044659E04FF0FF3404F10104DB
S11341380198FFF703FA0646FFF786FA0028F5D137
S1134148B6F1FF3F08BF4FF0FF3447D018F001071E
S113415801BF049B1A1D04921B680EBF039300221F
S11341680392002D16DC1AE005F1FF351FB9039BF5
S113417803F8016B039304F101040198FFF7DEF9D6
S11341880646431C18BF0123002DD4BF002303F0A7
S1134198010323B13046FFF757FA0028E4D030462C
S11341A80199FFF775FDCFB94FF00002039B1A7010
S11341B814E048F080020095019804A94FF00A031E
S11341C8FFF776FD044609E048F08002009501985F
S11341D804A94FF01003FFF76BFD0446002C0FDA17
S11341E8029A131C18BF0123B4F1FF3F0CBF1C46ED
S11341F843F00104002C08BF4FF0FF32029207E09D
S113420818F0010F02BF029B01330293A3441BE67B
S1134218029805B0BDE8F08F00B503B400F008F8C3
S113422803BC02B4694609BE00F004F801BC00BD31
S10B4238704700BF704700BF8E
S113424005000000000000008025000000000000C0
S113425000000000000000003031323334353637BE
S113426038396162636465663031323334353637E8
S10B427038394142434445463C
S10B4278008000000048E80189
S90321716A
